:10000000B6C0CFC0CEC0CDC0CCC0CBC0CAC0C9C0A6
:10001000C8C0C7C0C6C0C5C0C4C0C3C0C2C0C1C0BC
:10002000C0C0BFC0BEC018C12BC141C10DC50CC5E9
:1000300078C178C209C508C507C506C505C504C588
:1000400003C502C5B1C11AC21CC243C2FBC340C230
:10005000F8C387C499C485C497C496C495C4B5C46D
:1000600053C14CC1F1C4F0C4EFC4EEC4EDC4ECC440
:10007000EBC4EAC4E9C4E8C4E7C4E6C4E5C4E4C424
:100080003AC124C126C1E0C427C129C134C136C147
:1000900029C1DAC436C1D8C4D7C436C126C128C1E3
:1000A0001B5B306D1B5B324A1B5B303B3066004193
:1000B00076725573623530302D312E37207465726B
:1000C0006D696E616C206D6F64650D0A00456E741C
:1000D00065722053572056657273696F6E204D61AB
:1000E0006A6F7220696E20686578205B005D3A2037
:1000F00000456E7465722053572056657273696FA0
:100100006E204D696E6F7220696E20686578205B85
:10011000005D3A20000D0A4F4B2C206D792053577B
:100120002076657273696F6E206973206E6F773AFF
:1001300020002028686578290D0A005265616479DD
:100140002E204A75737420636C6F73652074686524
:10015000207465726D696E616C2E204E6F20726521
:10016000736574206E65656465642E0D0A00112444
:100170001FBECFE5D4E0DEBFCDBF10E0A0E6B0E00B
:10018000E2E6F0E102C005900D92AC36B107D9F776
:1001900011E0ACE6B0E001C01D92A03AB107E1F772
:1001A0003CC52ECFFF920F931F93CF93DF93182F51
:1001B000EB01CB0101978D51914028F0C2E0D0E0D6
:1001C00080EC809377008BE1C8D69BE1F92E812FDC
:1001D000C4D6F1268D2F9927182FBFD6F1268C2F44
:1001E000BCD6FC268EE0B9D68EE0F826ABD620979A
:1001F00059F006E710E0F8018081AFD6F80181914F
:100200008F01F8262197B9F78F2DA7D6DF91CF91CF
:100210001F910F91FF9008955F926F927F928F923E
:100220009F92AF92BF92CF92DF92EF92FF920F9385
:100230001F93CF93DF93582EE1E06E2E80917600CE
:100240009927AA27BB27FC013197ED31F10508F06A
:10025000FBC3ED5EFF4F099481E08093760010921E
:10026000770088E08093780089E0A1E6B0E0E9E7D4
:10027000F0E00D9001928A95E1F70BE010E0E9C300
:1002800080917700883921F48091780071D51BC165
:100290008E3929F4809178008093600014C18F39E1
:1002A00009F011C180917800809375000CC1809194
:1002B00077009927AA27BB27FC01E058F040E032DD
:1002C000F10508F0C1C3E05DFF4F0994E0909E0185
:1002D0001DC0E0909F011AC072E3E72E1BC069E1C8
:1002E000E62E18C080D5E82E11C0E09060000EC048
:1002F000E09075000BC052E0E52E0CC041E0E42E0A
:1003000009C03CE8E32E06C0EE2404C02FEFE2163D
:1003100009F49AC303E010E010927700E0927800AD
:1003200098C360917700862F9927AA27BB27B82FFB
:10033000AA279927882770917800272F33274427E9
:100340005527A90133272227822B932BA42BB52BCA
:1003500020917900332744275527542F432F322FDC
:100360002227822B932BA42BB52B20917A003327A5
:1003700044275527822B932BA42BB52B80937100F8
:1003800090937200A0937300B093740067FF04C051
:1003900081E08093700002C01092700070936F0033
:1003A00081E080936E008FC0A89839D58091780045
:1003B0009927ACD502E010E080EC80937700CC2444
:1003C000DD2480917A00813318F080E380937A00F5
:1003D00080917B00882319F481E080937B008091D9
:1003E0007A009927C816D90608F033C3ABD5A89868
:1003F0008091790099278AD50894C11CD11C8091DD
:100400007E0029D580917B00992780D580917F003F
:1004100022D580917B00992779D5A89A8091800078
:100420001AD5E82E80917B00992770D580918100A4
:1004300012D5782E90917D00933039F480917C0014
:10044000E81669F4109277000AC080917C00781653
:1004500011F410927700992311F490937700809112
:100460007700882331F4A89880917A00C82EDD2483
:10047000B6CFBDD484E190E049D5B1CF3FD5A89A9D
:1004800022C080917900E7D480917A00E4D48091F1
:100490007B00E1D480917C00DED4809178008823B9
:1004A00029F480917700992731D50DC0C6E9FC2E3B
:1004B00001C0FA9460E070E080E090EF03D580FF27
:1004C00002C0FF20B1F702E010E010927700C1C235
:1004D0006624882499245401B6E9FB2E80917A0081
:1004E000843018F484E080937A0080917A0081321D
:1004F00018F080E280937A008091710090917200F0
:1005000090936D0080936C00809177009927D82F8D
:10051000CC27809178009927C82BD92B81E0C9314D
:10052000D80720F002E010E080EC91C20BD570906B
:100530007900EE24872D9927809590959C01217054
:10054000307080FF94C0CC24DD24CC16DD0608F08A
:1005500073C106E710E0662031F0C0FE04C0809150
:100560007B00886002C080917B0075D4809171000F
:10057000909172009BD4F80182856DD490917E0099
:10058000F8018285981799F0809071009090720020
:10059000A0907300B09074008FEF9FEFA0E0B0E0E8
:1005A00088229922AA22BB227092790003C082E09D
:1005B00080937900C7D4662019F482E090E0A6D435
:1005C00080917900992782FF19C0F6E9FF2E6620F5
:1005D00031F0C0FE04C080917D00886002C080912F
:1005E0007D0039D4C40162D480E035D4FA9490916E
:1005F0007E008917B9F4FF2051F714C083FF0EC0A5
:10060000E6E9FE2E01C0FA9460E070E080E090EF31
:1006100059D480FF07C0FF20B1F704C080917A0051
:10062000992774D4662011F0C0FE13C08091710028
:1006300090917200A0917300B09174000196A11D79
:10064000B11D8093710090937200A0937300B093DA
:100650007400FF2011F470E8E72E0894C11CD11C2F
:100660000F5F1F4FCC16DD0608F475CFE5C069019A
:100670002C173D0708F08CC006E710E063D480918A
:1006800070008823A9F08091710090917200892BED
:1006900021F080916E00882359F08DE4DCD380E056
:1006A000DAD380916F00D7D380E0D5D310926E005B
:1006B000662031F0C0FE04C080917B00886002C0DB
:1006C00080917B00C8D38091710090917200EED32D
:1006D000F8018285C0D390917E00F8018285981739
:1006E00089F08090710090907200A0907300B0909B
:1006F00074008FEF9FEFA0E0B0E088229922AA2239
:10070000BB2206C080917900807880618093790057
:10071000662011F1C0FE33C080917100909172008B
:10072000A0917300B09174000196A11DB11D80933A
:10073000710090937200A0937300B0937400A07046
:10074000B0708F5F9F4FA040B040C9F480916F00A0
:100750008F5F80936F0013C0809171009091720041
:10076000A0917300B09174000196A11DB11D8093FA
:10077000710090937200A0937300B093740008947A
:10078000C11CD11C0F5F1F4FCC16DD0608F476CFBD
:10079000D9D38091790087FF4FC080917C005BD3D3
:1007A00080916C0090916D0081D380E054D36620DD
:1007B00019F481E090E0AAD366E9F62E80917900E1
:1007C00085FF24C081149104A104B104F9F0D5017E
:1007D000C40181709070A070B070892B21F080915D
:1007E0007D00886002C080917D0035D3C4015ED356
:1007F00080E031D3FA9490917E00891711F4FF20A4
:1008000031F7FF20C9F450E8E52E16C086FF10C06E
:1008100001C0FA9460E070E080E090EF53D380FF75
:1008200002C0FF20B1F7FF2039F441E8E42E04C0F4
:1008300080917A0099276AD302E010E0E092770075
:1008400008C16624809177009927D82FCC27809102
:1008500078009927C82BD92BE0907900F1E0C931B5
:10086000DF0710F0C8E1D1E0CC24DD24CC16DD0692
:1008700008F06EC008E710E065D38091700088230F
:10088000A9F08091710090917200892B21F08091E4
:100890006E00882359F08DE4DED280E0DCD28091B6
:1008A0006F00D9D280E0D7D210926E00662029F076
:1008B000C0FE03C08E2D886001C08E2DCCD28091E9
:1008C000710090917200F2D280E0C5D2D8018C9371
:1008D000662011F1C0FE33C08091710090917200CA
:1008E000A0917300B09174000196A11DB11D809379
:1008F000710090937200A0937300B0937400A07085
:10090000B0708F5F9F4FA040B040C9F480916F00DE
:100910008F5F80936F0013C080917100909172007F
:10092000A0917300B09174000196A11DB11D809338
:10093000710090937200A0937300B09374000894B8
:10094000C11CD11C0F5F1F4FCC16DD0608F494CFDD
:100950008E010D5F1F4F10927700CA58DF4F1A8229
:1009600078C08091770077D28091780074D280919E
:10097000790071D280917A006ED203E010E010927B
:1009800077001092780065C008E710E0C0E0D0E082
:1009900023E0F22ED8018D918D015DD2E82E809159
:1009A0007700992721968C179D0711F4E092780023
:1009B00085E090E0ABD2FA94F7FEECCF04E010E0D3
:1009C000109277001092790044C0E0907800709007
:1009D0007900FF24CF2D80917700F81600F585E08F
:1009E00090E094D2C71580F0FE1470F40F2D1127FB
:1009F0000A581F4FEC2FFF27EA58FF4F84812BD254
:100A0000F8018283F39406C0EC2FFF27EA58FF4FCA
:100A1000848121D2CF5F80917700C81700F3FE1444
:100A200040F4EF2DFF27E858FF4F1192F394FE1486
:100A3000E0F3EF2DFF278F010D5F1F4F109277001E
:100A4000EA58FF4F128205C002E010E089EC809363
:100A50007700B801852DA6DBDF91CF911F910F9113
:100A6000FF90EF90DF90CF90BF90AF909F908F90CE
:100A70007F906F905F900895EF92FF920F931F9376
:100A8000CF93C1E0FC2EB2E0EB2E1FEF8111FE2CC4
:100A900081E086D2C82F8D30D1F18A30C1F10C2F80
:100AA00000530A3038F08C2F8154863018F0805271
:100AB000863020F51F3F09F410E08C2F4ED20A300B
:100AC00028F41295107F1C0F105317C08C2F8154DF
:100AD000212F3327863048F4A4E0220F331FAA9534
:100AE000E1F71C2F120F175308C0F4E0220F331F39
:100AF000FA95E1F71C2F120F1755EA9481E050D2B6
:100B0000C82F8D3021F08A3011F0EE2041F6CD3023
:100B100011F0CA3009F4FA94FF2019F081E040D2B4
:100B2000FACF812F9927CF911F910F91FF90EF90CE
:100B300008958BE112D285E410D20895CF93C82F87
:100B400080EA90E01CD28FEA90E019D28DEC90E020
:100B500016D280919E0140E150E066E770E099274F
:100B600044D286E790E0FDD18DEE90E008D28C2F44
:100B700083DF8F3F11F080939E01DBDF81EF90E0F8
:100B8000FED180919F0140E150E066E770E0992737
:100B90002CD286E790E0E5D181E191E0F0D18C2F75
:100BA0006BDF8F3F11F080939F01C3DF60919F0146
:100BB00081E090E00FD260919E0182E090E00AD245
:100BC00064E180E090E006D285E191E0D8D18091A7
:100BD0009E0140E150E066E770E0992706D286E783
:100BE00090E0BFD18EE2B9D180919F01803110F4A5
:100BF00080E3B3D180919F0140E150E066E770E06F
:100C00009927F3D186E790E0ACD182E391E0B7D1A8
:100C10008BE391E0B4D1CF910895CFE5D4E0DEBF6E
:100C2000CDBFDD24BD2CCD2CC0E0D0E07E018CD129
:100C30007FD1A09AA89A939A969AC29AC398C59877
:100C40008B9A8E9ABA9ABB9ABD9ABC9878948AE08D
:100C500080939F0182E080939E0180E090E0B2D17A
:100C6000843151F481E090E0ADD180939F0182E026
:100C700090E0A8D180939E0181E092D104C080E0F1
:100C80008FD1112321F58B3119F411E0082FF7CF03
:100C90008D3019F08A3009F065C02196BB2039F4F7
:100CA0008A3029F49DE0D91611F401E0B02ED82E37
:100CB000BB2029F0C430D105F9F681E004C0C23070
:100CC000D105D1F68B2D3ADFC0E0D0E0D5CF113081
:100CD00021F4C82E082712E0D2CF123031F40827B1
:100CE0009927F82EEE2413E0CACF133031F40827E9
:100CF0009927E82AF92A14E0C2CF143041F40827D2
:100D00008E3009F0B9CF15E0C0E0D0E0B8CF153093
:100D1000A1F4CE15DF0534F591E0C831D90714F5FB
:100D20000827FE01EA58FF4F80832196A895CE152B
:100D3000DF0509F0A4CF16E0A2CF163099F4801792
:100D400039F41E141F0424F4A8958C2D65DA0AC00A
:100D500080EB8093760081EC8093770062E070E016
:100D60008C2D20DAEE24FF24DD24CD2CE70184CF66
:100D700010929D01843048F081E080939D018CE0C9
:100D800080936A008CE090E00895833048F070987A
:100D9000699A689A83E080936A0083E090E00895FE
:100DA000823048F07098699A689882E080936A006F
:100DB00082E090E00895813041F470986998689AD3
:100DC00080936A0081E090E00895882341F4709850
:100DD0006898699880936A0080E090E0089581E0C7
:100DE00090E00895089580916A00992708952DB1A3
:100DF0001DB8C5988CE590E0FC013197F1F7C59AD4
:100E00000197F1F7C5982DB90895C29A8CE590E045
:100E10000197F1F7C29884E190E078D008958B9A19
:100E20008E9ABA9AC29ABB9AC398BD9AC59893985B
:100E3000969884E190E06AD080919D01882329F4FE
:100E400081E58DB980916A0093DFC29884E190E0DA
:100E50005DD0DBDF0895CF93DF93482F20E830E0AB
:100E600080919D01882331F44FB9779BFECF8FB1DC
:100E7000992719C0C598ACE5B0E0C0E0D0E0842F58
:100E8000822311F0C39A01C0C398CD010197F1F7F5
:100E9000B499322BC59ACD010197F1F7C5982695E3
:100EA00071F7832F9927DF91CF9108950F931F93A7
:100EB0008C01812F9927CFDF802FCDDF99271F91BC
:100EC0000F910895EF92FF920F931F937B018C0176
:100ED000892F9927AA27BB27BEDFC801AA27BB27CE
:100EE000BADFBB27A12F902F8F2DB5DF8E2DB3DF5B
:100EF00099271F910F91FF90EF900895939A969ADA
:100F00001DB8C29AC398C598C29A0895CF93DF932B
:100F10009C01892B51F0A4E7B3E0C0E0D0E0CD0103
:100F20000197F1F721503040D1F7DF91CF9108952B
:100F300088E190E02FE00FB6F894A89581BD0FBE30
:100F400021BD0895A895089510BC81E090E089B96D
:100F500088E18AB986E880BD08955D9BFECF8CB993
:100F60000895CF93DF93EC018881882329F089913C
:100F7000F4DF88818823D9F7DF91CF910895CF934B
:100F8000DF93EC01FC0121968491882331F0E5DFA9
:100F9000FE01219684918823D1F7DF91CF910895A6
:100FA000CF93C82F5F9904C0C111CCDF5F9BFCCFEA
:100FB0008CB19927CF9108955F9B03C08CB15F9945
:100FC000FDCF0895E199FECF9FBB8EBBE09A992794
:100FD0008DB30895E199FECF9FBB8EBB6DBB0FB65D
:100FE000F894E29AE19A0FBE0895E62FF72F2E2F7C
:100FF0003F2F423074F0453264F4642F77271DD0C0
:10100000805D8A330CF0895D8193862F972F00973E
:10101000A1F7932F822F108200C0DC01FC01019008
:101020000020E9F73297AE17BF0730F47C9160815A
:10103000708331976D93F7CF0895AA1BBB1B51E1C5
:1010400007C0AA1FBB1FA617B70710F0A61BB70B38
:10105000881F991F5A95A9F780959095BC01CD01DD
:021060000895F1
:0C106200014156524953505F320001001A
:00000001FF
